:020000040000FA
:020000002028B6
:020008000900ED
:10001000000030340134913400008F34E93424344A
:10002000000001348634523400000000000000005B
:100030000000013493343A34000000000000000056
:1000400003016F20831285010730990083162C303D
:100050008500FF3095007F3081008312B2010920B6
:1000600059200A2059200B20592068200D205920A2
:100070000E2059200F205920682020306F20051DA8
:100080004928112059201220592013205920682076
:100090005028192059201A2059201B205920682047
:1000A00004308316960083128B0105088B156300BC
:1000B0002F28B0000830B1005E288514B00D320D35
:1000C0008500B10B5D288514000000008501080043
:1000D00005160830B100B10B6B2805120800B400FA
:0C00E000B301B30B7128B40B71280800A9
:02400E00C43FAD
:1042000043006F0070007900720069006700680069
:1042100074002000320030003100320020004A00DB
:104220006F0068006E0020004F0027004C006F00F8
:104230007500670068006C0069006E0020002000B7
:00000001FF
